:1000000012C021C068C01FC01EC01DC01CC01BC0C4
:100010001AC032C118C017C016C015C014C013C012
:1000200012C011C010C011241FBECFE5D4E0DEBF46
:10003000CDBF10E0A0E6B0E001C01D92A437B1072B
:10004000E1F76ED015C3DCCF982F8FE084BB15BAD3
:10005000992319F4A898A9980895913039F4A8988B
:10006000A99A80EE9EE2A0E0B0E008C0923079F458
:10007000A89AA99880EC94EDA1E0B0E080936F007D
:1000800090937000A0937100B09372000895933024
:1000900071F4A89AA99A80EC97E2A9E0B0E0809365
:1000A0006F0090937000A0937100B0937200089558
:1000B000882311F4AA9808C0813019F4AA98AB9A41
:1000C0000895823019F4AA9AAB980895833011F4F8
:1000D000AA9AAB9A08951F920F920FB60F9211240D
:1000E0008F939F93AF93BF9380916400909165002D
:1000F000A0916600B09167000196A11DB11D80938B
:10010000640090936500A0936600B0936700BF9170
:10011000AF919F918F910F900FBE0F901F901895E8
:100120008CE085BF80E88BBF8ABF83B7826083BFC6
:1001300089B7816089BFD0D182E086DFF894789456
:1001400081E0BED180EA9FE00197F1F7FFCFEF9207
:10015000FF920F931F93F8948823C1F481E8B0D1E4
:1001600082E5B4D180ECACD16091640070916500FF
:10017000809166009091670021EB33E040E050E011
:1001800016D220ED37E040E050E02EC0833099F4E5
:1001900087E896D187E49AD186EC92D16091640089
:1001A0007091650080916600909167002DEA32E0C1
:1001B00040E050E014C0813001F58DE881D182E447
:1001C00085D18CEC7DD16091640070916500809147
:1001D00066009091670022E632E040E050E0E7D10F
:1001E00028EE33E040E050E021D2209364003093C9
:1001F00065004093660050936700609164007091C1
:10020000650080916600909167002FEF30E040E03C
:1002100050E0CDD120916F0030917000409171007D
:100220005091720003D279018A01E0926B00F09242
:100230006C0000936D0010936E00D801C70122E09E
:10024000880F991FAA1FBB1F2A95D1F78E0D9F1DDE
:10025000A01FB11FACD010926900109268001092DC
:1002600064001092650010926600109267001F9162
:100270000F91FF90EF9008951F920F920FB60F927B
:1002800011242F933F934F935F936F937F938F939B
:100290009F93AF93BF93EF93FF9386E082BF8091CC
:1002A00068009091690001969093690080936800BE
:1002B00080559F4041F5F89480916A00882309F4A5
:1002C00046DF80916A00813009F441DF80916A0045
:1002D000833009F43CDF80916A008F5F80936A006D
:1002E000843010F010926A0080916A00823019F414
:1002F00083E080936A0080916A00DADE80E197E211
:100300000197F1F77894FF91EF91BF91AF919F9191
:100310008F917F916F915F914F913F912F910F90AE
:100320000FBE0F901F901895EF92FF920F931F939F
:100330009C0168EE73E066D1182F092FC90168EEA1
:1003400073E060D1662311F480E302C0862F805DE4
:10035000BDD0812F902F64E670E054D1F82EE92EA5
:10036000812F902F64E670E04DD1662311F480E375
:1003700002C0862F805DAAD08F2D9E2D6AE070E08E
:1003800041D1362F8F2D9E2D6AE070E03BD1182F82
:10039000332311F480E302C0832F805D97D0812F37
:1003A000805D94D01F910F91FF90EF9008950F936F
:1003B0001F939C0164E670E025D1182F092FC90115
:1003C00064E670E01FD1662311F480E302C0862F3B
:1003D000805D7CD0812F902F6AE070E013D1362FA2
:1003E000812F902F6AE070E00DD1182F332311F484
:1003F00080E302C0832F805D69D0812F805D66D04D
:100400001F910F9108951F93282F64E6EFD0192FA5
:10041000822FECD0882311F480E301C0805D56D098
:10042000812F6AE0E3D0282F812FE0D0192F2223DB
:1004300011F480E302C0822F805D48D0812F805D5F
:1004400045D01F9108951F93282F6AE0CFD0382FF1
:10045000822FCCD0192F332311F480E302C0832FD5
:10046000805D34D0812F805D31D01F910895805DF3
:100470002DD008959AE69A95F1F7909892B3807FDF
:100480009F70982B92BB929A85E08A95F1F792988B
:10049000089592B3282F207F9F70292B22BB929A18
:1004A00025E0922F9A95F1F7929892B38295807FEA
:1004B0009F70982B92BB929A2A95F1F79298089583
:1004C0009AE69A95F1F79098E4DF08959AE69A955E
:1004D000F1F7909ADEDF08950F931F9381B3806F39
:1004E00081BB889A899A8A9A80E991E028EC30E069
:1004F000F9013197F1F70197D9F780E3BBDF80E28B
:100500009EE40197F1F780E3B5DF00EA1FE0C80140
:100510000197F1F780E3AEDF88E2ACDF88E2D0DF5D
:100520008CE0CEDF81E0CCDFC8010197F1F786E0F7
:10053000C7DF1F910F910895CF93DF93EC0102C0A5
:100540002196C4DF88818823D9F7DF91CF91089560
:10055000CF93DF93EC0104C0FE0184912196B6DFB6
:1005600088818823C9F7DF91CF9108950F931F9356
:10057000CF93DF938C01862F90E08770907023E0FB
:10058000880F991F2A95E1F780649ADFC0E0D0E0D8
:10059000F801EC0FFD1FE4918E2F98DF2196C830F3
:1005A000D105B1F7DF91CF911F910F910895629F0F
:1005B000D001739FF001829FE00DF11D649FE00D5B
:1005C000F11D929FF00D839FF00D749FF00D659FBC
:1005D000F00D9927729FB00DE11DF91F639FB00DBB
:1005E000E11DF91FBD01CF0111240895991B79E088
:1005F00004C0991F961708F0961B881F7A95C9F7B3
:1006000080950895AA1BBB1B51E107C0AA1FBB1F01
:10061000A617B70710F0A61BB70B881F991F5A958E
:10062000A9F780959095BC01CD010895A1E21A2EFD
:10063000AA1BBB1BFD010DC0AA1FBB1FEE1FFF1F86
:10064000A217B307E407F50720F0A21BB30BE40BD6
:10065000F50B661F771F881F991F1A9469F760951D
:100660007095809590959B01AC01BD01CF010895D7
:04067000F894FFCF2C
:00000001FF
